:020000040000FA
:04000000F0303A287A
:040004000034003490
:08000800A000030EA100831209
:100010008B1C32288B1032181428B21C3228643002
:10002000010203183128182800001628172818285C
:1000300019281A281B281C281D281E281F283210A2
:10004000B214A810031005190314AA0DA90DA80DC8
:10005000B10B322832152A08AF002908AE00280853
:10006000AD00B21081010B11210E8300A00E200EF5
:02007000090085
:0C007400203084008001840A80300402E7
:10008000031C3C281230B100CB2183160C308505AF
:1000900087018312850187010730990000309A009B
:1000A000103083168E008312603083168F00831207
:1000B00000308316910000008312C830831681003F
:1000C000831231309000003083168C008312103080
:1000D0008B00BD1B7128851971286400851D6D2852
:1000E000B522A02281018E018F010B118B100B1004
:1000F0008C018B17892032199F20B40B872803109D
:1001000085190314BA0DF0303A0203193321FB228A
:100110007A286400321808000B1D08000B11B21079
:1001200032141230B100051D9A28331483160113BE
:10013000831208003310831601178312080032114E
:100140000130B7008B132030370783169B001C1437
:100150001A088312A400A500C030A5061030370786
:1001600083169B001C141A088312A3000030370763
:1001700083169B001C141A088312A2008B17331CD1
:10018000C72822090339A200A309A409A509220846
:100190002D02031D2D2923082E02031D2D292408BD
:1001A0002F02031D2D2901303702031DDC283E18C4
:1001B000DC283E143F14ED2102303702031DE528F0
:1001C000BE18E528BE143F14FC2103303702031D7E
:1001D000EE283E19EE283E153F140822043037025F
:1001E000031DF728BE19F728BE153F141422053049
:1001F0003702031D00293E1A00293E163F14202213
:1002000006303702031D0929BE1A0929BE163F14FC
:100210002F2207303702031D12293E1B12293E17D9
:100220003F143E2208303702031D1B29BE1B1B2929
:10023000BE173F14492209303702031D24295D18D7
:1002400024295D143F1454220A303702031D2D293E
:10025000DD182D29DD143F145F22B70A0B30370259
:1002600003180800A2280130B600B400B500B7009A
:1002700085018701B2139D228920B40B4C290310FC
:1002800085190314BA0DF0303A0203197329B50B1E
:100290004C299630B5007F21321D3C293211331C88
:1002A00056292D090339AD00AE09AF092F1CB21331
:1002B0002F1C3C29B21B3C292E183C29B2178B134A
:1002C00020303707BC002F08BB00B621103037079D
:1002D000BC002E08BB00B62100303707BC002D083B
:1002E000BB00B6218B1785018701B70AB601013023
:1002F000B5000B303702031C3C29A0220800013056
:10030000370203196B2202303702031970220330BF
:100310003702031975220430370203197A22053097
:10032000370203197F22063037020319842207306F
:100330003702031989220830370203198E22093047
:100340003702031993220A30370203199822080052
:100350003F1C08003F101030BC003E08BB00B62117
:100360003030BC005D08BB00B62108008B133B0891
:1003700083161C159A0083123C0883169B00553087
:100380009D00AA309D009C1464009C18C4291C1177
:1003900083128B170800831600309B001C141A0868
:1003A0008312BD00831610309B001C141A088312A0
:1003B000BE00831630309B001C141A088312DD0027
:1003C000FF30C800CA15CB15CC15CD15CE15CF15ED
:1003D000D015D115D215D3150800C130BE05FF3098
:1003E000DD055F140130C405C0000030C200BD1837
:1003F0005E14BD18DE140800C230BE05FF30DD05F6
:100400005F140230C405C0000030C2005E10080056
:10041000C430BE05FF30DD055F140630C405C000E2
:100420000030C2005E100800C830BE05FF30DD0598
:100430005F140A30C405C0000030C2005E1008001E
:10044000D030BE05FF30DD055F141130C405C0009B
:100450000030C200BD185E14BD18DE140800E03084
:10046000BE05FF30DD055F142130C405C00020301B
:10047000C200BD185E14BD18DE1408007F30BE0532
:100480000030DD05DF143030C505C1000030C30089
:100490000800BF30BE050030DD05DF14C030C505E3
:1004A000C1000030C30008003F30BE050130DD054B
:1004B000DF14D030C505C1000030C30008003F3054
:1004C000BE050230DD05DF14B030C505C1000030C7
:1004D000C3000800080010308506003087060800B9
:1004E0002030850600308706080021308506003060
:1004F0008706080022308506003087060800103085
:10050000850602308706080010308506043087060D
:100510000800003085062130870608000030850677
:100520001830870608000030850619308706080055
:10053000003085062930870608003E186B22080027
:100540003E18ED21BE18FC213E190822BE191422C6
:100550003E1A2022BE1A2F223E1B3E22BE1B4922DB
:100560005D185422DD185F220800B601B401B50100
:100570003D1CBD2ABD01BD14BF2ABD013D143D086F
:10058000B6006400C32AC42AC52AC62AC72AFF3077
:10059000B51B8500B51F8501B40BC12AB50BC12A57
:1005A0000310B60CB608031DC12A0030BC003D087C
:1005B000BB00B621080005125C180516DC1C85126C
:1005C000DC1885165C1D05105C190514DC1D8510F2
:1005D000DC1985145C1E87105C1A8714DC1E071159
:1005E000DC1A07155C1F07105C1B0714DC1F871241
:1005F000DC1B871608008F08031908008F0178306C
:100600008E00C80F3F2DC80A4208430403190E2B61
:100610004208C600C2014308C700C301441C352B71
:10062000461C262BCA1C172BCA014A15432B4A1DF0
:100630001C2BCA01CA15432BCA1D212BCA014A16FD
:10064000432B4A1E432BCA01CA14432B4A1D2B2B92
:10065000CA014A16432BCA1D302BCA014A16432B26
:100660004A1E432BCA01CA14432BCA1C3A2BCA0187
:100670004A15432B4A1D3F2BCA01CA15432B4A1E5C
:10068000432BCA014A15C41C6A2BC61C5B2BCB1C0E
:100690004C2BCB014B15782B4B1D512BCB01CB1584
:1006A000782BCB1D562BCB014B16782B4B1E782B62
:1006B000CB01CB14782B4B1D602BCB014B16782B29
:1006C000CB1D652BCB014B16782B4B1E782BCB010A
:1006D000CB14782BCB1C6F2BCB014B15782B4B1DE0
:1006E000742BCB01CB15782B4B1E782BCB014B15E4
:1006F000441D9F2B461D902BCC1C812BCC014C15EF
:10070000AD2B4C1D862BCC01CC15AD2BCC1D8B2BD2
:10071000CC014C16AD2B4C1EAD2BCC01CC14AD2B0B
:100720004C1D952BCC014C16AD2BCC1D9A2BCC011E
:100730004C16AD2B4C1EAD2BCC01CC14AD2BCC1CD0
:10074000A42BCC014C15AD2B4C1DA92BCC01CC15E9
:10075000AD2B4C1EAD2BCC014C15C41DD52BC61D8D
:10076000C62BCD1CB72BCD014D155E13E32B4D1DB4
:10077000BC2BCD01CD15E32BCD1DC12BCD014D16CD
:10078000E32B4D1EE32BCD01CD14E32B4D1DCB2BC5
:10079000CD014D16E32BCD1DD02BCD014D16E32BF6
:1007A0004D1EE32BCD01CD14E32BCD1CDA2BCD0157
:1007B0004D15E32B4D1DDF2BCD01CD15E32B4D1E2C
:1007C000E32BCD014D155E1B0C2C441E0C2C461E3C
:1007D000FD2BCE1CEE2BCE014E151A2C4E1DF32BED
:1007E000CE01CE151A2CCE1DF82BCE014E161A2C8A
:1007F0004E1E1A2CCE01CE141A2C4E1D022CCE01E8
:100800004E161A2CCE1D072CCE014E161A2C4E1E3B
:100810001A2CCE01CE141A2CCE1C112CCE014E1542
:100820001A2C4E1D162CCE01CE151A2C4E1E1A2C2B
:10083000CE014E15C41E412CC61E322CCF1C232CBB
:10084000CF014F154F2C4F1D282CCF01CF154F2C0A
:10085000CF1D2D2CCF014F164F2C4F1E4F2CCF01EB
:10086000CF144F2C4F1D372CCF014F164F2CCF1DBF
:100870003C2CCF014F164F2C4F1E4F2CCF01CF14C5
:100880004F2CCF1C462CCF014F154F2C4F1D4B2CFE
:10089000CF01CF154F2C4F1E4F2CCF014F15DE1916
:1008A0007A2CDE187A2C451E7A2C471E6B2CD01C15
:1008B0005C2CD0015015882C501D612CD001D01516
:1008C000882CD01D662CD0015016882C501E882CE8
:1008D000D001D014882C501D702CD0015016882CBB
:1008E000D01D752CD0015016882C501E882CD0019C
:1008F000D014882CD01C7F2CD0015015882C501D72
:10090000842CD001D015882C501E882CD001501575
:10091000DE19B32CDE18B32CC51EB32CC71EA42CB5
:10092000D11C952CD1015115C12C511D9A2CD101EE
:10093000D115C12CD11D9F2CD1015116C12C511E96
:10094000C12CD101D114C12C511DA92CD10151169A
:10095000C12CD11DAE2CD1015116C12C511EC12C60
:10096000D101D114C12CD11CB82CD1015115C12CED
:10097000511DBD2CD101D115C12C511EC12CD1014D
:100980005115DE19ED2CDE18ED2C451FED2C471FFF
:10099000DE2CD21CCF2CD2015215DE13FB2C521DA3
:1009A000D42CD201D215FB2CD21DD92CD201521637
:1009B000FB2C521EFB2CD201D214FB2C521DE32C1B
:1009C000D2015216FB2CD21DE82CD2015216FB2C60
:1009D000521EFB2CD201D214FB2CD21CF22CD201C1
:1009E0005215FB2C521DF72CD201D215FB2C521E96
:1009F000FB2CD2015215DE19282DDE18282DDE1B06
:100A0000282DC51F282DC71F192DD31C0A2DD30132
:100A10005315362D531D0F2DD301D315362DD31D50
:100A2000142DD3015316362D531E362DD301D31456
:100A3000362D531D1E2DD3015316362DD31D232DB8
:100A4000D3015316362D531E362DD301D314362D14
:100A5000D31C2D2DD3015315362D531D322DD3010B
:100A6000D315362D531E362DD3015315A82140081A
:100A7000C4004108C5005E18DE145E1CDE10480884
:100A8000C9000C304A05031D05120C304B05031D2F
:100A900085120C304C05031D05100C304D05031D4F
:100AA00085100C304E05031D87100C304F05031DBB
:100AB00007110C305005031D07100C305105031DA4
:100AC00087120C305205031D07120C305305031D0D
:100AD000871149080E020318992D12304A05031D8B
:100AE000051612304B05031D851612304C05031DEB
:100AF000051412304D05031D851412304E05031DDB
:100B0000871412304F05031D071512305005031DC1
:100B1000071412305105031D871612305205031DAC
:100B2000071612305305031D8715FF3048020319BD
:100B300008008F08031D0800892049080E02031CC5
:100B4000992D18304A05031D051206304A05031D6C
:100B5000051618304B05031D851206304B05031D85
:100B6000851618304C05031D051006304C05031D75
:100B7000051418304D05031D851006304D05031D65
:100B8000851418304E05031D871006304E05031DD1
:100B9000871418304F05031D071106304F05031D3C
:100BA000071518305005031D071006305005031DAA
:100BB000071418305105031D871206305105031D17
:100BC000871618305205031D071206305205031D03
:100BD000071618305305031D871106305305031DF2
:040BE000871508006D
:084000000E000300070001009F
:02400E00CC33B1
:10420000010003000300030003000200020002009B
:104210000200000000000000000003000300030093
:10422000410000000000000000000000000000004D
:104230000000C000C000C000C000C000C000C0003E
:10424000FF00C300F300CF00FF00C300F300CF0066
:10425000FF00C300F300CF00FF00C300F300CF0056
:104260000000FF00FF00FF00FF00FF00FF00FF0055
:10427000FF00FF00FF00FF00FF00FF00FF00FF0046
:10428000FF000300FF00FF00FF00FF00FF00FF0032
:10429000FF00FF00FF00FF00FF00FF00FF00FF0026
:1042A000FF00C000FF00FF00FF00FF00FF00FF0055
:1042B000FF00FF00FF00FF00FF00FF00FF00FF0006
:1042C000FF00FF00FF00FF00FF00FF00FF00FF00F6
:1042D000FF00FF00FF00FF00FF00FF00FF00FF00E6
:1042E000FF00FF00FF00FF00FF00FF00FF00FF00D6
:1042F000FF00FF00FF00FF00FF00FF00FF00AA001B
:00000001FF
